:020000020000FC
:100000000DC0189518951895189518951895189568
:10001000B3C01895189518951895C8C000E00EBF84
:100020000FED0DBF00E808B901E007B906EC06B90D
:1000300003E00EBD0DEF0DBD0FE80CBD01E00CB9E6
:100040004FEE00EF0ABB0BBB07E007BBDD27C4E0A8
:1000500000E3402E502E602E702E70E68827789494
:10006000EE24FF2430E1359A339A369A44D0332374
:10007000E9F733983598F694E794F694E79404EF0B
:1000800011E054D01694079416940794A72FBB2719
:100090000D921C921197EE24FF2420E10D91E00EA9
:1000A0000D91F01E8395803111F4A0E688272A95E2
:1000B000A9F712968395803111F4A0E688277A2F4C
:1000C00024E0F694E7942A95E1F73DD0A4E0BB271D
:1000D000012D02950F70002319F40FEF0D9301C04D
:1000E0001BD0012D906418D09F7B002D029514D059
:1000F000002D12D0B5CF00E205BF8895002705BFBF
:10010000089528E0C098000F10F4C19A01C0C1986A
:10011000C09A2A95B9F70895E8EBF1E00F70E00F67
:10012000FB1F049196FD0F7D0D930895222420E17D
:100130001695079510F41E0C2F1C279417940794FE
:100140002A95B1F7089520E1222411240024FF27E5
:10015000EE0CFF1C001C111C221C2A9509F40895AA
:10016000E3E002910D5F03FD00830081005D07FD68
:100170000083E030B1F7ECCF0F930FB70F930BB3C1
:10018000006F0BBBC2980991BCDFC29A0BB3006F22
:1001900004230BBB440F10F04FEEC4E00DEF0DBD78
:1001A0000FE80CBD0F910FBF0F91189504B1E00E31
:1001B00005B1F01E3A95189530F32AA2E1A424F275
:0201C00020A07D
:00000001FF
